:0C000000830100308A0004288301BD2B1E
:10072A008312A0009B2BFA308312A0238312A0030A
:10073A00200F982B08008312A0000430A100533028
:10074A00A200A20BA62BA10BA42BA00BA22B080084
:10075A008312A1008312A003200FAF2BB92B3D30C7
:10076A00A200A203220FB62BA103210FB42B08006B
:10077A00831285010730990083169F0183120510A1
:10078A00831605108312CE233E30A023CE236300A6
:10079A0004285A308312E3233230A0006C30AD2390
:1007AA001A30E3231330A0000530AD231730E323BA
:1007BA000930A0000D30AD231A30E32B8312A000BC
:1007CA00FA2B0514000000000000000000000000E1
:1007DA0000000000000000000510000000000000FA
:1007EA00000000000000000000008312A003200F98
:0407FA00E62B0800E2
:02400E00843FED
:00000001FF
